:0E0000000C9434000C9400000C9400000C943E
:10000E0000000C9400000C9400000C9400000C9462
:10001E0000000C9400000C9400000C9400000C9452
:10002E0000000C9400000C9400000C9400000C9442
:10003E0000000C9451000C9400000C9400000C94E1
:10004E0000000C9400000C9400000C9400000C9422
:10005E0000000C9400000C940000F894EE27EFBB07
:10006E00F1E0F5BFE5BF8DE0A2E0BB27ED938A95E9
:10007E00E9F780E098E0A0E0B1E0ED930197E9F7B1
:10008E00E0E0EEBBEFEFEDBFE8E0EEBFC0E0D3E0A7
:10009E000C946C006A937A93AA93BA93EA93FA93A8
:1000AE00EFB7EA93A0E0B3E00E94FE00EF5FFF4FD0
:1000BE006F4F7F4F0E940301E991EFBFF991E991D4
:1000CE00B991A9917991699118952C97E0E0E093F7
:1000DE000003E0930103E0930203E0930303EC8338
:1000EE00ED83EE83EF83E8EEF3E060E070E00E94D4
:1000FE000D01E0E8E0936100E0E0E0936100E4B917
:10010E00E5B9E7B9E8B9EAB9EBB9E3E0E4BDEBE08C
:10011E00E5BDE0E0E6BDECE7E7BDE0E0E8BDE0937D
:10012E008000E0938100E0938500E0938400E093EB
:10013E008700E0938600E0938900E0938800E093C7
:10014E008B00E0938A00E093B600E093B000E0935A
:10015E00B100E093B200E093B300E093B400E1E0AD
:10016E00E0936E00E0E0E0936F00E0937000E093A8
:10017E006900EDBBE0936800E093C100E0E8E0BFEA
:10018E00E0E0E0937B00E0937F00E0937A00ECBD2B
:10019E00E093BC007894E0910003F091010360912C
:1001AE00020370910303E887F9876A877B87AC8126
:1001BE00BD818E819F810E94F900DF01CB010E94DB
:1001CE0008010E94120160F4E5B1A0E2EA27E5B948
:1001DE00E885F9856A857B85EC83FD836E837F8355
:1001EE00DACFFFCFEA1BFB0B680B790B0895ED916D
:1001FE00FD916D917D9108957E936E93FE93EE9396
:10020E000895E881F9816A817B810895E883F983F5
:10021E006A837B830895EA17FB07680779070895B9
:00000001FF
